 battdrvr

 Timestamp is 4fb04cbe (Mon May 14 12:07:26 2012)

 Preferred load address is 10000000

 Start         Length     Name                   Class
 0001:00000000 00000004H .CRT$XCA                CODE
 0001:00000004 00000004H .CRT$XCZ                CODE
 0001:00000008 00000004H .CRT$XIA                CODE
 0001:0000000c 00000004H .CRT$XIZ                CODE
 0001:00000010 00000004H .CRT$XPA                CODE
 0001:00000014 00000004H .CRT$XPZ                CODE
 0001:00000018 00000004H .CRT$XTA                CODE
 0001:0000001c 00000004H .CRT$XTZ                CODE
 0001:00000020 000000a4H .rdata                  CODE
 0001:000000c4 00000025H .rdata$debug            CODE
 0001:000000ec 00001510H .text                   CODE
 0001:00001600 00000104H .xdata                  CODE
 0001:00001704 00000014H .idata$2                CODE
 0001:00001718 00000014H .idata$3                CODE
 0001:0000172c 0000008cH .idata$4                CODE
 0001:000017b8 0000000cH .idata$6                CODE
 0001:000017d0 000000dcH .edata                  CODE
 0002:00000000 0000008cH .idata$5                DATA
 0002:0000008c 00000008H .data                   DATA
 0002:000000a0 000000f8H .bss                    DATA
 0003:00000000 00000170H .pdata                  DATA

  Address         Publics by Value              Rva+Base       Lib:Object

 0000:00000000       ___safe_se_handler_table   00000000     <absolute>
 0000:00000000       ___safe_se_handler_count   00000000     <absolute>
 0001:00000000       __xc_a                     10001000     corelib0:crt0init.obj
 0001:00000004       __xc_z                     10001004     corelib0:crt0init.obj
 0001:00000008       __xi_a                     10001008     corelib0:crt0init.obj
 0001:0000000c       __xi_z                     1000100c     corelib0:crt0init.obj
 0001:00000010       __xp_a                     10001010     corelib0:crt0init.obj
 0001:00000014       __xp_z                     10001014     corelib0:crt0init.obj
 0001:00000018       __xt_a                     10001018     corelib0:crt0init.obj
 0001:0000001c       __xt_z                     1000101c     corelib0:crt0init.obj
 0001:0000003c       ??_C@_1BM@KBMAGFOO@?$AAP?$AAd?$AAd?$AAB?$AAu?$AAf?$AAf?$AAe?$AAr?$AAS?$AAi?$AAz?$AAe?$AA?$AA@ 1000103c     battdrvr_lib:battdrvr.obj
 0001:00000058       ??_C@_1BK@GMCBNGHD@?$AAP?$AAo?$AAl?$AAl?$AAI?$AAn?$AAt?$AAe?$AAr?$AAv?$AAa?$AAl?$AA?$AA@ 10001058     battdrvr_lib:battdrvr.obj
 0001:00000074       ??_C@_1CA@NFABIDNC@?$AAP?$AAo?$AAl?$AAl?$AAP?$AAr?$AAi?$AAo?$AAr?$AAi?$AAt?$AAy?$AA2?$AA5?$AA6?$AA?$AA@ 10001074     battdrvr_lib:battdrvr.obj
 0001:00000094       ??_C@_1DA@IBFGCKKH@?$AAS?$AAY?$AAS?$AAT?$AAE?$AAM?$AA?1?$AAB?$AAa?$AAt?$AAt?$AAe?$AAr?$AAy?$AAA?$AAP?$AAI?$AAs?$AAR?$AAe?$AAa?$AAd?$AAy?$AA?$AA@ 10001094     battdrvr_lib:battdrvr.obj
 0001:000000ec       BatteryPDDInitialize       100010ec f   battdrvr.obj
 0001:000000f4       BatteryPDDDeinitialize     100010f4 f   battdrvr.obj
 0001:000000f8       BatteryPDDResume           100010f8 f   battdrvr.obj
 0001:000000fc       BatteryPDDPowerHandler     100010fc f   battdrvr.obj
 0001:00000100       BatteryPDDGetStatus        10001100 f   battdrvr.obj
 0001:00000120       BatteryPDDGetLevels        10001120 f   battdrvr.obj
 0001:00000128       BatteryPDDSupportsChangeNotification 10001128 f   battdrvr.obj
 0001:00000130       BatteryThreadProc          10001130 f   battdrvr_lib:battdrvr.obj
 0001:00000218       Init                       10001218 f   battdrvr_lib:battdrvr.obj
 0001:0000055c       Deinit                     1000155c f   battdrvr_lib:battdrvr.obj
 0001:0000063c       IOControl                  1000163c f   battdrvr_lib:battdrvr.obj
 0001:00000ba0       PowerDown                  10001ba0 f   battdrvr_lib:battdrvr.obj
 0001:00000bb4       PowerUp                    10001bb4 f   battdrvr_lib:battdrvr.obj
 0001:00000bdc       Open                       10001bdc f   battdrvr_lib:battdrvr.obj
 0001:00000be0       Close                      10001be0 f   battdrvr_lib:battdrvr.obj
 0001:00000be8       Read                       10001be8 f   battdrvr_lib:battdrvr.obj
 0001:00000c00       Write                      10001c00 f   battdrvr_lib:battdrvr.obj
 0001:00000c18       Seek                       10001c18 f   battdrvr_lib:battdrvr.obj
 0001:00000c20       DllMain                    10001c20 f   battdrvr_lib:battdrvr.obj
 0001:00000c38       BatteryAPIStopwatch        10001c38 f   battdrvr_lib:battapi.obj
 0001:00000d14       BatteryAPIGetSystemPowerStatusEx2 10001d14 f   battdrvr_lib:battapi.obj
 0001:00000f58       BatteryAPIGetSystemPowerStatusEx 10001f58 f   battdrvr_lib:battapi.obj
 0001:00000f94       BatteryAPIGetLifeTimeInfo  10001f94 f   battdrvr_lib:battapi.obj
 0001:00001048       BatteryAPINotifyOfTimeChange 10002048 f   battdrvr_lib:battapi.obj
 0001:000010cc       EventModify                100020cc f   coredll:COREDLL.dll
 0001:000010dc       WaitForSingleObject        100020dc f   coredll:COREDLL.dll
 0001:000010ec       PowerPolicyNotify          100020ec f   coredll:COREDLL.dll
 0001:000010fc       CeSetThreadPriority        100020fc f   coredll:COREDLL.dll
 0001:0000110c       DeleteCriticalSection      1000210c f   coredll:COREDLL.dll
 0001:0000111c       LocalFree                  1000211c f   coredll:COREDLL.dll
 0001:0000112c       CloseHandle                1000212c f   coredll:COREDLL.dll
 0001:0000113c       CreateThread               1000213c f   coredll:COREDLL.dll
 0001:0000114c       LocalAlloc                 1000214c f   coredll:COREDLL.dll
 0001:0000115c       RegCloseKey                1000215c f   coredll:COREDLL.dll
 0001:0000116c       RegQueryValueExW           1000216c f   coredll:COREDLL.dll
 0001:0000117c       OpenDeviceKey              1000217c f   coredll:COREDLL.dll
 0001:0000118c       CreateEventW               1000218c f   coredll:COREDLL.dll
 0001:0000119c       InitializeCriticalSection  1000219c f   coredll:COREDLL.dll
 0001:000011ac       OpenEventW                 100021ac f   coredll:COREDLL.dll
 0001:000011bc       GetLastError               100021bc f   coredll:COREDLL.dll
 0001:000011cc       LeaveCriticalSection       100021cc f   coredll:COREDLL.dll
 0001:000011dc       EnterCriticalSection       100021dc f   coredll:COREDLL.dll
 0001:000011ec       SetLastError               100021ec f   coredll:COREDLL.dll
 0001:000011fc       CeSetPowerOnEvent          100021fc f   coredll:COREDLL.dll
 0001:0000120c       DisableThreadLibraryCalls  1000220c f   coredll:COREDLL.dll
 0001:0000121c       GetTickCount               1000221c f   coredll:COREDLL.dll
 0001:0000122c       SystemTimeToFileTime       1000222c f   coredll:COREDLL.dll
 0001:0000123c       GetLocalTime               1000223c f   coredll:COREDLL.dll
 0001:0000124c       FileTimeToSystemTime       1000224c f   coredll:COREDLL.dll
 0001:00001360       _DllMainCRTStartup         10002360 f   corelib0:pegdmain.obj
 0001:0000148c       _cexit                     1000248c f   corelib0:cexit.obj
 0001:000014a8       _initterm                  100024a8 f   corelib0:crt0dat.obj
 0001:000014dc       _cinit                     100024dc f   corelib0:crt0dat.obj
 0001:00001510       __security_init_cookie     10002510 f   corelib0:seccinit.obj
 0001:0000156c       memcpy                     1000256c f   corelib1:COREDLL.dll
 0001:0000157c       memcmp                     1000257c f   corelib1:COREDLL.dll
 0001:0000158c       memset                     1000258c f   corelib1:COREDLL.dll
 0001:0000159c       __C_specific_handler       1000259c f   corelib1:COREDLL.dll
 0001:000015ac       _XcptFilter                100025ac f   corelib1:COREDLL.dll
 0001:000015bc       free                       100025bc f   corelib1:COREDLL.dll
 0001:000015cc       __security_gen_cookie2     100025cc f   corelib1:COREDLL.dll
 0001:000015dc       InterlockedExchange        100025dc f   coredll:COREDLL.dll
 0001:000015ec       TerminateProcess           100025ec f   coredll:COREDLL.dll
 0001:00001704       __IMPORT_DESCRIPTOR_COREDLL 10002704     coredll:COREDLL.dll
 0001:00001718       __NULL_IMPORT_DESCRIPTOR   10002718     coredll:COREDLL.dll
 0002:00000000       __imp_EventModify          10003000     coredll:COREDLL.dll
 0002:00000004       __imp_WaitForSingleObject  10003004     coredll:COREDLL.dll
 0002:00000008       __imp_PowerPolicyNotify    10003008     coredll:COREDLL.dll
 0002:0000000c       __imp_CeSetThreadPriority  1000300c     coredll:COREDLL.dll
 0002:00000010       __imp_DeleteCriticalSection 10003010     coredll:COREDLL.dll
 0002:00000014       __imp_LocalFree            10003014     coredll:COREDLL.dll
 0002:00000018       __imp_CloseHandle          10003018     coredll:COREDLL.dll
 0002:0000001c       __imp_CreateThread         1000301c     coredll:COREDLL.dll
 0002:00000020       __imp_LocalAlloc           10003020     coredll:COREDLL.dll
 0002:00000024       __imp_RegCloseKey          10003024     coredll:COREDLL.dll
 0002:00000028       __imp_RegQueryValueExW     10003028     coredll:COREDLL.dll
 0002:0000002c       __imp_OpenDeviceKey        1000302c     coredll:COREDLL.dll
 0002:00000030       __imp_CreateEventW         10003030     coredll:COREDLL.dll
 0002:00000034       __imp_InitializeCriticalSection 10003034     coredll:COREDLL.dll
 0002:00000038       __imp_OpenEventW           10003038     coredll:COREDLL.dll
 0002:0000003c       __imp_GetLastError         1000303c     coredll:COREDLL.dll
 0002:00000040       __imp_LeaveCriticalSection 10003040     coredll:COREDLL.dll
 0002:00000044       __imp_EnterCriticalSection 10003044     coredll:COREDLL.dll
 0002:00000048       __imp_SetLastError         10003048     coredll:COREDLL.dll
 0002:0000004c       __imp_CeSetPowerOnEvent    1000304c     coredll:COREDLL.dll
 0002:00000050       __imp_DisableThreadLibraryCalls 10003050     coredll:COREDLL.dll
 0002:00000054       __imp_GetTickCount         10003054     coredll:COREDLL.dll
 0002:00000058       __imp_SystemTimeToFileTime 10003058     coredll:COREDLL.dll
 0002:0000005c       __imp_GetLocalTime         1000305c     coredll:COREDLL.dll
 0002:00000060       __imp_FileTimeToSystemTime 10003060     coredll:COREDLL.dll
 0002:00000064       __imp_memcpy               10003064     corelib1:COREDLL.dll
 0002:00000068       __imp_memcmp               10003068     corelib1:COREDLL.dll
 0002:0000006c       __imp_memset               1000306c     corelib1:COREDLL.dll
 0002:00000070       __imp___C_specific_handler 10003070     corelib1:COREDLL.dll
 0002:00000074       __imp__XcptFilter          10003074     corelib1:COREDLL.dll
 0002:00000078       __imp_free                 10003078     corelib1:COREDLL.dll
 0002:0000007c       __imp___security_gen_cookie2 1000307c     corelib1:COREDLL.dll
 0002:00000080       __imp_InterlockedExchange  10003080     coredll:COREDLL.dll
 0002:00000084       __imp_TerminateProcess     10003084     coredll:COREDLL.dll
 0002:00000088       \177COREDLL_NULL_THUNK_DATA 10003088     coredll:COREDLL.dll
 0002:0000008c       __security_cookie          1000308c     corelib0:seccinit.obj
 0002:00000090       __security_cookie_complement 10003090     corelib0:seccinit.obj
 0002:000000a0       _exitflag                  100030a0     corelib0:cexit.obj
 0002:000000a4       v_imsStart                 100030a4     <common>
 0002:000000a8       v_fStopwatchRunning        100030a8     <common>
 0002:000000b0       v_ftLastChange             100030b0     <common>
 0002:000000b8       v_cmsPreviousCpuUsage      100030b8     <common>
 0002:000000bc       v_fOnExternalPower         100030bc     <common>
 0002:000000c0       v_cmsUsed                  100030c0     <common>
 0002:000000e0       gcsPddBuffer               100030e0     <common>
 0002:00000100       gBatteryContext            10003100     <common>
 0002:00000140       ghevResume                 10003140     <common>
 0002:00000144       gpfnBatteryPddIOControl    10003144     <common>
 0002:00000160       gcsBattery                 10003160     <common>
 0002:00000174       gpPddBufferTemp            10003174     <common>
 0002:00000178       gpPddBuffer                10003178     <common>
 0002:0000017c       gdwPddBufferSize           1000317c     <common>
 0002:00000180       gfExiting                  10003180     <common>
 0002:00000184       ghtBattery                 10003184     <common>
 0002:00000188       __onexitend                10003188     <common>
 0002:0000018c       __onexitbegin              1000318c     <common>
 0002:00000190       g_pcsExit                  10003190     <common>
 0002:00000194       _pRawDllMain               10003194     <common>

 entry point at        0001:00001360

 Static symbols

 0001:00001264       _DllMainCRTStartupHelper   10002264 f   corelib0:pegdmain.obj
 0001:00001390       doexit                     10002390 f   corelib0:cexit.obj
